:10000000000000308A002B28A501A400FF30A407BF
:10001000031CA507031C26280330A300DF30122091
:100020000628A301E83EA200A309FC30031C1B28FC
:10003000A20703181828A2070000A30F18282218E7
:100040002128A21C252800002528080083138312DC
:100050000313000008000130A500F4308A010520D8
:10006000831685013F3086008701880183128A1537
:100070000A1209258A110A12861841288A150A12BD
:1000800012208A110A12861848288A110A12FE2E96
:100090008A110A128626A101A0018A110A12B32A26
:1000A000003021078A005B30200703188A0AA00A63
:1000B0000319A10A820001340034003400340034F2
:1000C000003400340034003400340234003400348E
:1000D000003400340034003400340034003404347C
:1000E0000034003400340034003400340034003470
:1000F0000034083400340034003400340034003458
:10010000003400340034103400340034003400343F
:10011000003400340034003400342034003400341F
:10012000003400340034003400340034003400342F
:10013000013400340034003400340034003400341E
:10014000003400340234003400340034003400340D
:1001500000340034003400340434003400340034FB
:1001600000340034003400340034003408340034E7
:1001700000340034003400340034003400340034DF
:1001800010340034003400340034003400340034BF
:10019000003400342034003400340034003400349F
:1001A00000340034003400340034013400340034AE
:1001B000003400340034003400340034003402349D
:1001C000003400340034003400340034003400348F
:1001D000003404340034003400340034003400347B
:1001E0000034003400340834003400340034003467
:1001F000003400340034003400341034003400344F
:10020000003400340034003400340034003420342E
:10021000003400340034003400340034003400343E
:10022000003400340134003400340034003400342D
:10023000003400340034003402340034003400341C
:10024000003400340034003400340034043400340A
:1002500000340034003400340034003400340034FE
:1002600008340034003400340034003400340034E6
:1002700000340034103400340034003400340034CE
:1002800000340034003400342034003400340034AE
:1002900000340034003400340034003400340134BD
:1002A00000340034003400340034003400340034AE
:1002B000003402340034003400340034003400349C
:1002C000003400340034043400340034003400348A
:1002D0000034003400340034003408340034003476
:1002E000003400340034003400340034003410345E
:1002F000003400340034003400340034003400345E
:10030000003420340034003400340034003400342D
:10031000003400340034003401340034003400343C
:10032000003400340034003400340034023400342B
:10033000003400340034003400340034003400341D
:100340000434003400340034003400340034003409
:1003500000340034083400340034003400340034F5
:1003600000340034003400341034003400340034DD
:1003700000340034003400340034003420340034BD
:1003800000340034003400340034003400340034CD
:1003900000340134003400340034003400340034BC
:1003A00000340034003402340034003400340034AB
:1003B0000034003400340034003404340034003499
:1003C0000034003400340034003400340034083485
:1003D000003400340034003400340034003400347D
:1003E000003410340034003400340034003400345D
:1003F000003400340034203400340034003400343D
:10040000003400340034003400340034013400344B
:10041000003400340034003400340034003400343C
:10042000023400340034003400340034003400342A
:100430000034003404340034003400340034003418
:100440000034003400340034083400340034003404
:1004500000340034003400340034003410340034EC
:1004600000340034003400340034003400340034EC
:1004700020340034003400340034003400340034BC
:1004800000340034003401340034003400340034CB
:1004900000340034003400340034023400340034BA
:1004A00000340034003400340034003400340434A8
:1004B000003400340034003400340034003400349C
:1004C0000034083400340034003400340034003484
:1004D000003400340034103400340034003400346C
:1004E000003400340034003400342034003400344C
:1004F000003400340034003400340034003400345C
:10050000013400340034003400340034003400344A
:100510000034003402340034003400340034003439
:100520000034003400340034043400340034003427
:100530000034003400340034003400340834003413
:10054000003400340034003400340034003400340B
:1005500010340034003400340034003400340034EB
:10056000003400342034B00ABF0A8A015020A600AB
:100570008A015020A7008A015020A8008A0150203B
:10058000A9008A015020AA008A015020AB008A01EC
:100590005020AC008A015020AD008A015020AE00EE
:1005A0008A015020AF003C303F028A110A12031D1D
:1005B000DA2ABF013F088A110A12031DE12AA101AC
:1005C000A001C0018A110A12061CE92A8A110A1226
:1005D000912F26088A110A12031DF02A320887007B
:1005E000260832028A110A12031DF82A32088700EF
:1005F000320826028A110A120318012B2608320239
:100600008700260832028A110A1203180A2B3208C0
:10061000260787000A308A01042040308700270817
:100620008A110A12031D162B33088700330827028C
:100630008A110A1203181F2B270833028700270884
:1006400033028A110A120318282B33082707870060
:100650000A308A0104204030870028088A110A12D3
:10066000031D342B34088700340828028A110A122B
:1006700003183D2B280834028700280834028A1109
:100680000A120318462B3408280787000A308A010B
:1006900004204030870029088A110A12031D522BBA
:1006A00035088700350829028A110A1203185B2BC6
:1006B000290835028700290835028A110A12031811
:1006C000642B3508290787000A308A01042040304E
:1006D00087002A088A110A12031D702B360887002A
:1006E00036082A028A110A120318792B2A083602C0
:1006F00087002A0836028A110A120318822B36084C
:100700002A0787000A308A010420403087002B081E
:100710008A110A12031D8E2B3708870037082B0217
:100720008A110A120318972B2B08370287002B080F
:1007300037028A110A120318A02B37082B078700EB
:100740000A308A010420403087002C088A110A12DE
:10075000031DAC2B3808870038082C028A110A12B6
:100760000318B52B2C08380287002C0838028A1190
:100770000A120318BE2B38082C0787000A308A019A
:100780000420403087002D088A110A12031DCA2B4D
:100790003908870039082D028A110A120318D32B51
:1007A0002D08390287002D0839028A110A12031810
:1007B000DC2B39082D0787000A308A0104204030DD
:1007C00087002E088A110A12031DE82B3A088700B9
:1007D0003A082E028A110A120318F12B2E083A0247
:1007E00087002E083A028A110A120318FA2B3A08D7
:1007F0002E0787000A308A010420403087002F0826
:100800008A110A12031D062C3B0887003B082F02A1
:100810008A110A1203180F2C2F083B0287002F0899
:100820003B028A110A120318182C3B082F07870075
:100830002430A300CA308A0112208030870087014B
:100840008A110A1286263D3030028A110A12031DCF
:100850002C2C8A110A12452CC00A323040028A110F
:100860000A12031D352C8A01B32A8A110A120619AD
:100870003C2C8A150A1279298A110A128618432CEF
:100880008A110A12FE2E8A01E22AC001BF01B001BC
:100890008A150A12C024A101A00101303C028A116C
:1008A0000A12031D552C0130B20002303C028A119D
:1008B0000A12031D5D2C0330B20003303C028A1182
:1008C0000A12031D652C0730B20004303C028A1165
:1008D0000A12031D6D2C0F30B20005303C028A1144
:1008E0000A12031D752C1F30B20006303C028A111B
:1008F0000A12031D7D2C3F30B20007303C028A11E2
:100900000A12031C852C3F30B20038303C028A1199
:100910000A12031C8D2C3E30B20007303C028A11B3
:100920000A12031D952C0130B30008303C028A11D5
:100930000A12031D9D2C0330B30009303C028A11BA
:100940000A12031DA52C0730B3000A303C028A119D
:100950000A12031DAD2C0F30B3000B303C028A117C
:100960000A12031DB52C1F30B3000C303C028A1153
:100970000A12031DBD2C3F30B3000D303C028A111A
:100980000A12031CC52C3F30B3000D303C028A1103
:100990000A12031DCD2C0130B4000E303C028A1126
:1009A0000A12031DD52C0330B4000F303C028A110B
:1009B0000A12031DDD2C0730B40010303C028A11EE
:1009C0000A12031DE52C0F30B40011303C028A11CD
:1009D0000A12031DED2C1F30B40012303C028A11A4
:1009E0000A12031DF52C3F30B40013303C028A116B
:1009F0000A12031CFD2C3F30B40013303C028A1154
:100A00000A12031D052D0130B50014303C028A1175
:100A10000A12031D0D2D0330B50015303C028A115A
:100A20000A12031D152D0730B50016303C028A113D
:100A30000A12031D1D2D0F30B50017303C028A111C
:100A40000A12031D252D1F30B50018303C028A11F3
:100A50000A12031D2D2D3F30B50019303C028A11BA
:100A60000A12031C352D3F30B50019303C028A11A3
:100A70000A12031D3D2D0130B6001A303C028A11C6
:100A80000A12031D452D0330B6001B303C028A11AB
:100A90000A12031D4D2D0730B6001C303C028A118E
:100AA0000A12031D552D0F30B6001D303C028A116D
:100AB0000A12031D5D2D1F30B6001E303C028A1144
:100AC0000A12031D652D3F30B6001F303C028A110B
:100AD0000A12031C6D2D3F30B6001F303C028A11F4
:100AE0000A12031D752D0130B70020303C028A1117
:100AF0000A12031D7D2D0330B70021303C028A11FC
:100B00000A12031D852D0730B70022303C028A11DE
:100B10000A12031D8D2D0F30B70023303C028A11BD
:100B20000A12031D952D1F30B70024303C028A1194
:100B30000A12031D9D2D3F30B70025303C028A115B
:100B40000A12031CA52D3F30B70025303C028A1144
:100B50000A12031DAD2D0130B80026303C028A1167
:100B60000A12031DB52D0330B80027303C028A114C
:100B70000A12031DBD2D0730B80028303C028A112F
:100B80000A12031DC52D0F30B80029303C028A110E
:100B90000A12031DCD2D1F30B8002A303C028A11E5
:100BA0000A12031DD52D3F30B8002B303C028A11AC
:100BB0000A12031CDD2D3F30B8002B303C028A1195
:100BC0000A12031DE52D0130B9002C303C028A11B8
:100BD0000A12031DED2D0330B9002D303C028A119D
:100BE0000A12031DF52D0730B9002E303C028A1180
:100BF0000A12031DFD2D0F30B9002F303C028A115F
:100C00000A12031D052E1F30B90030303C028A1134
:100C10000A12031D0D2E3F30B90031303C028A11FB
:100C20000A12031C152E3F30B90031303C028A11E4
:100C30000A12031D1D2E0130BA0032303C028A1107
:100C40000A12031D252E0330BA0033303C028A11EC
:100C50000A12031D2D2E0730BA0034303C028A11CF
:100C60000A12031D352E0F30BA0035303C028A11AE
:100C70000A12031D3D2E1F30BA0036303C028A1185
:100C80000A12031D452E3F30BA0037303C028A114C
:100C90000A12031C4D2E3F30BA0037303C028A1135
:100CA0000A12031D552E0130BB0038303C028A1158
:100CB0000A12031D5D2E0330BB0039303C028A113D
:100CC0000A12031D652E0730BB003A303C028A1120
:100CD0000A12031D6D2E0F30BB003B303C028A11FF
:100CE0000A12031D752E1F30BB003C303C028A11D6
:100CF0000A12031D7D2E3F30BB0001303C028A11D9
:100D00000A12031D842EBE0A8A01B32A0D303E0248
:100D10008A110A12031D8E2E0130BE0001303E02E0
:100D20008A110A12031D962E0130880002303E02FD
:100D30008A110A12031D9E2E0230880003303E02E3
:100D40008A110A12031DA62E0430880004303E02C8
:100D50008A110A12031DAE2E0830880005303E02AB
:100D60008A110A12031DB62E1030880006303E028A
:100D70008A110A12031DBE2E2030880007303E0261
:100D80008A110A12031DC62E4030880008303E0228
:100D90008A110A12031DCE2E8030880009303E02CF
:100DA0008A110A12031CD52E880109303E028A11CD
:100DB0000A12031DDD2E313085000A303E028A11F1
:100DC0000A12031DE52E323085000B303E028A11D7
:100DD0000A12031DED2E343085000C303E028A11BC
:100DE0000A12031DF52E3830850009303E028A11A3
:100DF0000A120318FD2E3030850008008A110A12ED
:100E0000061C052F8A110A12912F320887000A301A
:100E10008A01042040308700330887000A308A01A5
:100E20000420403087003408870009308A010420FC
:100E300040308700350887000A308A01042040309E
:100E40008700360887000A308A0104204030870076
:100E5000370887000A308A010420403087003808AC
:100E600087000A308A010420403087003908870053
:100E70000A308A010420403087003A0887000A308F
:100E80008A010420403087003B0887002830A300F7
:100E9000FA308A0112208030870087018A150A12F1
:100EA00012203D3030028A110A12031D592F8A0187
:100EB000452CC00AB10A323040028A110A12031DC1
:100EC000622FB00A323031028A110A1203186B2FD6
:100ED0008A150A128A20333031028A110A12031C41
:100EE000742F8A150A120221323040028A110A1226
:100EF000031D7B2FC001653031028A110A12031CC9
:100F0000822FB1018A110A12861C882F8A01E22AD7
:100F10008A110A1206198F2F8A150A1279298A0155
:100F2000FE2E87010A308A010420403087008701A5
:100F30000A308A01042040308700870109308A0185
:100F400004204030870087010A308A0104204030A5
:100F5000870087010A308A0104204030870087011A
:100F60000A308A0104204030870087010A308A0154
:100F700004204030870087010A308A010420403075
:100F8000870087010A308A010420403087008701EA
:100F90002830A300FA308A011220803087008701B0
:100FA0008A150A1212203D3030028A110A12031DDE
:100FB000DB2F8A01452CC00AB10A323040028A1167
:100FC0000A12031DE42FB00A323031028A110A12CC
:100FD0000318ED2F8A150A128A20333031028A1144
:100FE0000A12031CF62F8A150A12022185013230DB
:100FF00040028A110A12031DFE2FC0016530310222
:101000008A150A12031C0528B1018A150A12861CCA
:101010000A28B0018A150A12861810288A01FE2EA5
:101020008A01E22A0D303E028A150A12031D1A288F
:101030000130BE0001303E028A150A12031D22282B
:101040000130880002303E028A150A12031D2A2848
:101050000230880003303E028A150A12031D32282E
:101060000430880004303E028A150A12031D3A2813
:101070000830880005303E028A150A12031D4228F6
:101080001030880006303E028A150A12031D4A28D5
:101090002030880007303E028A150A12031D5228AC
:1010A0004030880008303E028A150A12031D5A2873
:1010B0008030880009303E028A150A12031C61281C
:1010C000880109303E028A150A12031D6928313051
:1010D00085000A303E028A150A12031D712832303B
:1010E00085000B303E028A150A12031D7928343020
:1010F00085000C303E028A150A12031D8128383003
:10110000850009303E028A150A12031889283030FA
:10111000850008000D303E028A150A12031D922830
:101120000130BE0001303E028A150A12031D9A28C2
:101130000130880002303E028A150A12031DA228DF
:101140000230880003303E028A150A12031DAA28C5
:101150000430880004303E028A150A12031DB228AA
:101160000830880005303E028A150A12031DBA288D
:101170001030880006303E028A150A12031DC2286C
:101180002030880007303E028A150A12031DCA2843
:101190004030880008303E028A150A12031DD2280A
:1011A0008030880009303E028A150A12031CD928B3
:1011B000880109303E028A150A12031DE1282130F8
:1011C00085000A303E028A150A12031DE9282230E2
:1011D00085000B303E028A150A12031DF1282430C7
:1011E00085000C303E028A150A12031DF9282830AA
:1011F000850009303E028A150A12031801292030A1
:10120000850008000D303E028A150A12031D0A29C6
:101210000130BE0001303E028A150A12031D122958
:101220000130880002303E028A150A12031D1A2975
:101230000230880003303E028A150A12031D22295B
:101240000430880004303E028A150A12031D2A2940
:101250000830880005303E028A150A12031D322923
:101260001030880006303E028A150A12031D3A2902
:101270002030880007303E028A150A12031D4229D9
:101280004030880008303E028A150A12031D4A29A0
:101290008030880009303E028A150A12031C512949
:1012A000880109303E028A150A12031D59290130AE
:1012B00085000A303E028A150A12031D6129023098
:1012C00085000B303E028A150A12031D692904307D
:1012D00085000C303E028A150A12031D7129083060
:1012E000850009303E028A150A1203187829850103
:1012F00008008A150A12061C7F298A01912FB00165
:10130000C001BF01A101A001320887000A308A0193
:10131000042040308700330887000A308A01042007
:1013200040308700340887000A308A0104204030AA
:101330008700350887000A308A0104204030870082
:10134000360887000A308A010420403087003708B9
:1013500087000A308A01042040308700380887005F
:101360000A308A01042040308700390887000530A0
:101370008A010420403087003A0887000A308A0139
:101380000420403087003B0887000A308A0104208F
:101390008030870087018A150A1249248A150A12AB
:1013A000861AD5298A150A12F6298A150A12061AEA
:1013B000DC298A150A12382C8A150A128619E329A3
:1013C0008A150A1209258A150A120619EA298A15A8
:1013D0000A1279298A150A12861CF0298A01E22A42
:1013E0008A150A128618F6298A01FE2E0130A500F8
:1013F000F4308A0105208A150A12861A022A8A15F3
:101400000A12F6298A150A12C02401303C028A15F4
:101410000A12031D0D2A0130B20002303C028A1567
:101420000A12031D152A0330B20003303C028A154C
:101430000A12031D1D2A0730B20004303C028A152F
:101440000A12031D252A0F30B20005303C028A150E
:101450000A12031D2D2A1F30B20006303C028A15E5
:101460000A12031D352A3F30B20007303C028A15AC
:101470000A12031C3D2A3F30B20038303C028A1564
:101480000A12031C452A3E30B20007303C028A157E
:101490000A12031D4D2A0130B30008303C028A15A0
:1014A0000A12031D552A0330B30009303C028A1585
:1014B0000A12031D5D2A0730B3000A303C028A1568
:1014C0000A12031D652A0F30B3000B303C028A1547
:1014D0000A12031D6D2A1F30B3000C303C028A151E
:1014E0000A12031D752A3F30B3000D303C028A15E5
:1014F0000A12031C7D2A3F30B3000D303C028A15CE
:101500000A12031D852A0130B4000E303C028A15F0
:101510000A12031D8D2A0330B4000F303C028A15D5
:101520000A12031D952A0730B40010303C028A15B8
:101530000A12031D9D2A0F30B40011303C028A1597
:101540000A12031DA52A1F30B40012303C028A156E
:101550000A12031DAD2A3F30B40013303C028A1535
:101560000A12031CB52A3F30B40013303C028A151E
:101570000A12031DBD2A0130B50014303C028A1541
:101580000A12031DC52A0330B50015303C028A1526
:101590000A12031DCD2A0730B50016303C028A1509
:1015A0000A12031DD52A0F30B50017303C028A15E8
:1015B0000A12031DDD2A1F30B50018303C028A15BF
:1015C0000A12031DE52A3F30B50019303C028A1586
:1015D0000A12031CED2A3F30B50019303C028A156F
:1015E0000A12031DF52A0130B6001A303C028A1592
:1015F0000A12031DFD2A0330B6001B303C028A1577
:101600000A12031D052B0730B6001C303C028A1558
:101610000A12031D0D2B0F30B6001D303C028A1537
:101620000A12031D152B1F30B6001E303C028A150E
:101630000A12031D1D2B3F30B6001F303C028A15D5
:101640000A12031C252B3F30B6001F303C028A15BE
:101650000A12031D2D2B0130B70020303C028A15E1
:101660000A12031D352B0330B70021303C028A15C6
:101670000A12031D3D2B0730B70022303C028A15A9
:101680000A12031D452B0F30B70023303C028A1588
:101690000A12031D4D2B1F30B70024303C028A155F
:1016A0000A12031D552B3F30B70025303C028A1526
:1016B0000A12031C5D2B3F30B70025303C028A150F
:1016C0000A12031D652B0130B80026303C028A1532
:1016D0000A12031D6D2B0330B80027303C028A1517
:1016E0000A12031D752B0730B80028303C028A15FA
:1016F0000A12031D7D2B0F30B80029303C028A15D9
:101700000A12031D852B1F30B8002A303C028A15AF
:101710000A12031D8D2B3F30B8002B303C028A1576
:101720000A12031C952B3F30B8002B303C028A155F
:101730000A12031D9D2B0130B9002C303C028A1582
:101740000A12031DA52B0330B9002D303C028A1567
:101750000A12031DAD2B0730B9002E303C028A154A
:101760000A12031DB52B0F30B9002F303C028A1529
:101770000A12031DBD2B1F30B90030303C028A1500
:101780000A12031DC52B3F30B90031303C028A15C7
:101790000A12031CCD2B3F30B90031303C028A15B0
:1017A0000A12031DD52B0130BA0032303C028A15D3
:1017B0000A12031DDD2B0330BA0033303C028A15B8
:1017C0000A12031DE52B0730BA0034303C028A159B
:1017D0000A12031DED2B0F30BA0035303C028A157A
:1017E0000A12031DF52B1F30BA0036303C028A1551
:1017F0000A12031DFD2B3F30BA0037303C028A1518
:101800000A12031C052C3F30BA0037303C028A15FF
:101810000A12031D0D2C0130BB0038303C028A1522
:101820000A12031D152C0330BB0039303C028A1507
:101830000A12031D1D2C0730BB003A303C028A15EA
:101840000A12031D252C0F30BB003B303C028A15C9
:101850000A12031D2D2C1F30BB003C303C028A15A0
:101860000A12031D352C3F30BB008A150A12792954
:10187000C0010130A500F4308A0105208A150A1242
:10188000061A452C8A150A12382CBE0A8A150A1225
:1018900079290D303E028A150A12031D512C0130A0
:1018A000BE0001303E028A150A12031D592C013078
:1018B000880002303E028A150A12031D612C023094
:1018C000880003303E028A150A12031D692C043079
:1018D000880004303E028A150A12031D712C08305C
:1018E000880005303E028A150A12031D792C10303B
:1018F000880006303E028A150A12031D812C203012
:10190000880007303E028A150A12031D892C4030D8
:10191000880008303E028A150A12031D912C80307F
:10192000880009303E028A150A12031C982C88018F
:1019300009303E028A150A12031DA02C01308500D1
:101940000A303E028A150A12031DA82C02308500B7
:101950000B303E028A150A12031DB02C043085009C
:101960000C303E028A150A12031DB82C083085007F
:1019700009303E028A150A120318BF2C850108009F
:10198000BC0A3D303C028A150A12031DC92C0130E5
:10199000BC0001303C028A150A12031DD02CB30191
:1019A00001303C028A150A12031DD72CB401013004
:1019B0003C028A150A12031DDE2CB50101303C02DF
:1019C0008A150A12031DE52CB60101303C028A1566
:1019D0000A12031DEC2CB70101303C028A150A12D1
:1019E000031DF32CB80101303C028A150A12031DB5
:1019F000FA2CB90101303C028A150A12031D012D8F
:101A0000BA0101303C028A150A12031D082DBB01E0
:101A100008000130B200B301B401B501B601B7014D
:101A2000B801B901BA01BB01A601A701A801A9012A
:101A3000AA01AB01AC01AD01AE01AF01B001C00123
:101A4000BF010130BE008701880180308700870117
:0A1A50000130BC00A101A001080054
:02400E00723FFF
:00000001FF
